:020000040000FA
:020000003228A4
:08000800A800030E8301A9000A
:10001000B8200030A8002208A80203192128FF30C8
:10002000A8002208A80203192A2805148510112106
:100030000510851014308E20831203138B108B173C
:1000400047280030DF200130DF200230DF2003307E
:10005000DF201A2805142308F820A720A720A720AE
:1000600005101A2883160130860008308500683094
:100070008F000F1D392800309B000B168B100113C9
:100080008B17831282308600003085000510B50181
:10009000B601B701B801B901C001C101C2013F21D8
:1000A0000301A8013608A80003013508A809A80221
:1000B000031D87280301A8013808A8000301370899
:1000C000A809A802031D87280301A8014008A80069
:1000D00003013908A809A802031D87280301A80104
:1000E0004208A80003014108A809A802031D8728A7
:1000F0003508DF203708DF203908DF204108DF20FE
:1001000005108514FF308E20051085104728051432
:10011000851032308E200510851047286400A60017
:10012000A430A700A70B9228A60B90280800640013
:10013000A6000230A700A70B9B28A60B9928080051
:10014000A600000000000000A60BA2280800FA305C
:100150008E20FA308E20FA308E20FA308E20FA303F
:100160008E20FA308E20FA308E20FA308E20080051
:10017000C320A100C320A200C320A300C320A40069
:10018000C320A50008000830A0000830A020AB0163
:100190001230A020000006182B140000AB0CA00B9E
:1001A000C82800001230A0201430AF00061CDA2846
:1001B000AF0BD628AB0C000000002B080800B000E5
:1001C0000830B100861009309720000000000000C0
:1001D000000000000000301C861030188614093022
:1001E0009720B00CB10BEB2886140930972008003B
:1001F000B0000830B10086130930972000000000DD
:100200000000000000000000301C86133018861724
:1002100009309720B00CB10B0429861709309720BC
:100220000800051512308E20051109308E20220895
:10023000AC002B212308AC002B212408AC002B217F
:100240002508AC002B2105152130972005115130D0
:100250008E20051108000230AD000830AE000515F3
:100260002130972005111730AC1B50309720AC0D72
:10027000AE0B2F29AC0DAC09AD0B2D2908000330B6
:10028000AA00FF30AE00851D3F29AE0B4329AA0B03
:100290004129851949290430AA00BE30AE008519CC
:1002A0003F29AE0B4F29AA0B4D29851D552900006A
:1002B000000000000000463097206E21B5076E2137
:1002C000B6076E21B7076E21B8076E21B9076E21F8
:1002D000C0076E21C1076E21C2070800C3010310C9
:1002E0000830A0008030AE00000000000000851D36
:1002F00082218519792928309720AE0CA00B74290A
:100300004308080003012E08C307851D852908003E
:02400E00103F61
:00000001FF
